S0130000666C6173686C6F616465722E737265638C
S113000000000320D904000045050000FD4A00005B
S1130010054B00000D4B0000154B000000000000D4
S11300200000000000000000000000004505000082
S1130030450500000000000045050000792400008B
S11300404505000045050000450500004505000084
S11300504505000045050000450500004505000074
S11300604505000045050000450500004505000064
S11300704505000045050000450500004505000054
S11300804505000045050000450500004505000044
S11300904505000045050000450500004505000034
S11300A0312500003D250000053500001135000014
S11300B045050000450500004505000059210000E4
S11300C0450500007921000045050000A921000034
S11300D045050000C9210000450500004505000054
S11300E045050000450500004505000045050000E4
S11300F045050000450500004505000045050000D4
S113010045050000450500004505000045050000C3
S113011045050000450500004505000045050000B3
S113012045050000450500004505000045050000A3
S1130130C95A0000815D0000450500004505000026
S1130140450500001D350000E921000045050000BB
S11301500922000045050000450500004505000092
S11301604505000045050000492500006D290000F3
S11301707929000085290000450500004505000097
S113018091290000450500004505000045050000D3
S11301904505000045050000450500004505000033
S11301A04505000045050000450500004505000023
S11301B04505000045050000450500004505000013
S11301C04505000045050000450500004505000003
S11303F0450500004505000045050000FFFFFFFF1F
S1130400FFFFFFFFFFFFFFFFFFFFFFFFFEFFFFFFF9
S113041010B5054C237833B9044B13B10448AFF33A
S113042000800123237010BDB804FF1F00000000EA
S1130430D460000008B5064B1BB106480649AFF36B
S113044000800648036813B1054B03B1984708BD03
S113045000000000D4600000BC04FF1FB404FF1FB0
S113046000000000154B002B08BF134B9D46A3F55D
S1130470803A00218B460F461348144A121A05F09D
S1130480C4FC0F4B002B00D098470E4B002B00D020
S113049098470020002104000D000D48002802D0D8
S11304A00C48AFF3008005F081FC2000290004F023
S11304B00DFB04F011FB00BF000008000000032046
S11304C00000000000000000B804FF1F300AFF1FF6
S11304D0000000000000000072B60E480E4988605B
S11304E00E4A0E4B0D4C0D4D0C4E0C4FB846B946F2
S11304F0BA46BB46BC460A4885460A4880470A486D
S113050080470A48804762B604480449084A90472D
S1130510FFF7FEBF0000000000ED00E00000000057
S113052000000320650D0000BD0C0000190D000043
S1130530CD4A000072B600F015FC00F0BFFB62B6B5
S1130540FFF790FFFFF7FEBF002A40F00280012072
S113055070472DE9F0001F46034603242340002B77
S113056000F00C800424E31A017001300824E141F6
S1130570013A00F03580013B7FF4F6AF042AC0F263
S1130580258000F01B80002F00F018800C460D46DB
S11305900E46102AC0F2048072C0103AFFF7F9BF69
S11305A00C2AC0F2048032C00C3AFFF7F9BF082AC3
S11305B0C0F2048012C0083AFFF7F9BF042AC0F25F
S11305C0058001600430043AFFF7F8BF002A00F008
S11305D00780017001300824E141013A7FF4F6AF4D
S11305E0F0BC0020704700BF4BB942B9002908BFD6
S11305F0002802D04FF0FF31084600F03BB882B02B
S1130600EC462DE9005000F01DF8DDF804E002B0DE
S11306100CBC70472DE97043069E14461D46804667
S1130620894600F029F804FB01F300FB0533A4FB21
S113063000451D44B8EB040469EB0505C6E9004513
S1130640BDE870832DE97043069E144680468946B2
S11306501D4600F05DF900FB05F504FB0153A0FB0A
S113066004451D44B8EB040469EB0505C6E90045DF
S1130670BDE87083704700BF00292DE9F00FC0F278
S11306809F800024002BC0F29680154606460F4634
S1130690002B3ED18A4257D9B2FA82F34BB1C3F14F
S11306A0200201FA03F720FA02F29D40174300FAF0
S11306B003F6290CB7FBF1F2330C01FB127CA8B250
S11306C043EA0C4700FB02F3BB4209D97F1902F14C
S11306D0FF3C80F00181BB4240F2FE80023A2F448D
S11306E0FF1AB7FBF1F3B6B201FB137146EA0141FD
S11306F000FB03F0884208D9491903F1FF3780F061
S1130700ED80884240F2EA80023B43EA0242002341
S113071003E08B420AD900231A461046194614B145
S1130720404261EB4101BDE8F00F7047B3FA83F832
S1130730B8F1000F40F084808B4202D3824200F271
S1130740DE8000230122E8E712B90123B3FBF2F5AE
S1130750B5FA85F2002A39D17F1B280C1FFA85FCD3
S11307600123B7FBF0F1320C00FB117742EA074793
S11307700CFB01F2BA4207D97F1901F1FF3802D20A
S1130780BA4200F2C1804146BF1AB7FBF0F2B6B2DA
S113079000FB127046EA00400CFB02FC844507D9BA
S11307A0401902F1FF3702D2844500F2AB803A4689
S11307B042EA0142B1E7E443524263EB430364E794
S11307C0404261EB41014FF0FF345BE79540C2F1D9
S11307D0200327FA03F1280C26FA03F39740B1FB10
S11307E0F0F81F433B0C00FB18111FFA85FC43EA89
S11307F001410CFB08F38B4206FA02F608D94919A9
S113080008F1FF3279D28B4277D9A8F10208294442
S1130810C91AB1FBF0F3BFB200FB131147EA014759
S11308200CFB03F2BA4207D97F1903F1FF3160D2FE
S1130830BA425ED9023B2F44BF1A43EA084390E709
S1130840C8F1200203FA08FC25FA02F343EA0C0C6F
S11308504FEA1C4921FA02F301FA08F720FA02F2DE
S1130860B3FBF9F1174309FB11333A0C1FFA8CFB64
S113087042EA03430BFB01FA9A4505FA08F008D94A
S113088013EB0C0301F1FF3235D29A4533D9023907
S11308906344CAEB0303B3FBF9F209FB1233BFB29F
S11308A047EA03470BFB02F9B94508D917EB0C07D4
S11308B002F1FF331BD2B94519D9023A674442EA1F
S11308C00145A5FB0001C9EB07078F424FF0000368
S11308D00AD305D02A4620E7624601E73B4614E7DF
S11308E006FA08F68642F5D26A1E002315E71A4670
S11308F0E5E70B46A0E71146CBE7904688E7434679
S113090042460AE7023A53E702392F443CE700BF64
S11309102DE9F00F144605460E46002B43D18A42BA
S113092053D9B2FA82F757B1C7F1200620FA06F676
S113093001FA07F302FA07F41E4300FA07F5210C43
S1130940B6FBF1F22B0C01FB1267A0B243EA074697
S113095000FB02F3B34209D9361902F1FF3780F0E4
S1130960F680B34240F2F380023A2644F61AB6FB0C
S1130970F1F3ADB201FB136145EA014100FB03F061
S1130980884208D9091903F1FF3680F0E2808842D1
S113099040F2DF80023B43EA02420023104619463C
S11309A0BDE8F00F70478B424AD8B3FA83F6002EA5
S11309B04DD18B4202D3824200F2D6800023012221
S11309C010461946BDE8F00F704712B90124B4FB74
S11309D0F2F4B4FA84F2002A7CD1091B260CA7B2E3
S11309E00123B1FBF6F02A0C06FB101142EA014187
S11309F007FB00F28A4207D9091900F1FF3C02D231
S1130A008A4200F2C3806046891AB1FBF6F2ADB2A5
S1130A1006FB121145EA014507FB02F7AF4208D96C
S1130A202C1902F1FF3180F09680A74240F29380A6
S1130A30023A42EA004210461946BDE8F00F7047F8
S1130A4000231A4610461946BDE8F00F7047C6F158
S1130A50200522FA05F4B3401C434FEA144821FA56
S1130A6005F301FA06F720FA05F5B3FBF8FC2F436A
S1130A7008FB1C333D0C1FFA84FA45EA03430AFBC6
S1130A800CF9994502FA06FB04D91B190CF1FF3243
S1130A906DD39446C9EB0303B3FBF8F508FB153398
S1130AA0BFB247EA03470AFB05F8B84504D93F1922
S1130AB005F1FF3361D31D4645EA0C4CACFB0B2317
S1130AC0C8EB07079F424FF0000549D345D0624663
S1130AD02B4663E79440C2F1200321FA03FC260C61
S1130AE020FA03F301FA02F5BCFBF6F843EA050128
S1130AF00B0C06FB18CCA7B243EA0C4C07FB08F31B
S1130B00634500FA02F509D91CEB040C08F1FF3225
S1130B103AD2634538D9A8F10208A444C3EB0C0CBB
S1130B20BCFBF6F389B206FB13CC41EA0C4107FB8C
S1130B3003F28A4207D9091903F1FF3022D28A420B
S1130B4020D9023B2144891A43EA084349E73A463B
S1130B500CE733461FE70A466BE7B0409042B6D233
S1130B600CF1FF32002319E73346324616E7994564
S1130B708FD9ACF1020C23448CE7B8459BD9023DD4
S1130B80274499E70346DEE79046C7E70238214445
S1130B903AE700BF08B5101A63EB0101024BD3E931
S1130BA00023FFF721FD08BDD804FF1F38B5044614
S1130BB00D460C4BD3E9002352EA030108D14FF44C
S1130BC07A7001F04BFC024600230649C1E9002378
S1130BD065700020207000220023C4E902232061F4
S1130BE038BD00BFD804FF1F38B504460D4643780E
S1130BF013F0FF0F08D072B64378013BDBB24370A9
S1130C000020207062B638BD11B3037813F0FF0FD3
S1130C1010D001F009FC02460B462569D4E9020113
S1130C20FFF7B8FF854215D272B60023237062B66F
S1130C30022038BDB1F1FF3F0ED072B6012303701C
S1130C4062B601F0F1FBC4E902012561032038BD5D
S1130C50022038BD032038BD032038BD4378DBB201
S1130C60FF2B07D072B643780133DBB2437062B610
S1130C7000207047012070470020704772B60022A0
S1130C80014B1A6062B67047D404FF1F72B6024B60
S1130C901A6801321A607047D404FF1F064B1B68A0
S1130CA0012B04D80022044B1A6062B67047024B31
S1130CB01A68013A1A607047D404FF1F0F4B104A98
S1130CC09A60104A104B9B1A1049914206D109E0D0
S1130CD008781070013B0131013201E009490B4AE7
S1130CE0002BF5D10A4A0B4B9B1A002102E011702C
S1130CF0013B0132002BFAD1704700BF00ED00E048
S1130D0000000000FC600000B46100000004FF1F4C
S1130D10B804FF1F300AFF1F114B4FF0FF32C3F816
S1130D208020C3F88420C3F88820C3F88C20C3F83B
S1130D309020C3F89420C3F89820C3F89C20C3F8EB
S1130D408021C3F88421C3F88821C3F88C21C3F817
S1130D509021C3F89421C3F89821C3F89C217047CB
S1130D6000E100E00A4B4CF22052DA814DF62812E1
S1130D70DA814FF4E9721A8003F52C339B7813F06F
S1130D80080F04D0034B9A7842F008029A70704717
S1130D900020054000D00740014B0360002070474D
S1130DA0A50D0000436A5A898282DA68023A4260D9
S1130DB05A6808498A4206D11B7A012B06D8064B89
S1130DC003600020704742F27570704742F27570FC
S1130DD0704700BF53544D50E10E000030B583B04E
S1130DE00446134B1B689B68C06D216E626A98476A
S1130DF0B8B90F4B1B681B69984798B904F11C05D7
S1130E002846616A102203F0E9FA284601A903F092
S1130E1011FB626E019B9A4205D1064B23600020B0
S1130E2003E002E001E042F27A7003B030BD00BF9B
S1130E301004FF1F3510000030B583B0044600F1E4
S1130E401C052846616A102203F0C8FA174B1B6878
S1130E509B68E06D1021626A984700BBE36D103314
S1130E60E365236E103B2366102B02D9104B2360DD
S1130E7019E01BB10F4B2360002014E00B4B1B68DF
S1130E801B69984760B9284601A903F0D3FA626E3A
S1130E90019B9A4205D1084B2360002003E002E045
S1130EA001E042F27A7003B030BD00BF1004FF1FAE
S1130EB0390E0000DD0D0000351000004268836823
S1130EC09A4208D9D21A42608366044B0360012314
S1130ED083600020704742F278707047351000003C
S1130EE010B582B00446436A5A6882611A68033AAC
S1130EF0826041688A4211D21B8993B902A901F820
S1130F00013D0A4802F08EF89DF807301BB92046CF
S1130F10FFF7D4FF07E042F2817004E042F27670FA
S1130F2001E042F2777002B010BD00BF3004FF1F31
S1130F3010B504461C3003F04BFA236E102B02D973
S1130F40034B236001E0034B2360002010BD00BF6E
S1130F50390E0000DD0D000010B50346044A126886
S1130F60D468C06D196E5A6EA0470028FFD010BD1A
S1130F701004FF1F42F21270704700BF08B5036EE1
S1130F8083604268934212D8426E12F0010F06D079
S1130F90C16D8269914202D1C360002008BDB0F8DE
S1130FA05A3013F0010F05D1FFF788FF08BD42F254
S1130FB0767008BD42F27C7008BD00BF08B50346D8
S1130FC0B0F85A2012F0010F02D000F011FE08BD53
S1130FD0034A12685269C06D196E904708BD00BF7C
S1130FE01004FF1F10B5054C20460021702204F0A8
S1130FF00CFF034B2360002010BD00BFF404FF1F4F
S1131000990D000010B50446C36D23B1406E04F180
S11310101801984701E042F27F70012803D120466D
S1131020FFF74CFF10BD022802D1FFF7DBFF0020C1
S113103010BD00BF38B5054600F15804436A0FCB14
S113104084E80F005A22012302E0E15C0A440133E0
S11310500F2BFAD995F85830D2B2934223D195F890
S11310605930072B22D8DFE803F004060A0E1216C3
S1131070041A002038BD2846FFF780FF38BD2846F3
S1131080FFF756FF38BD2846FFF766FF38BD2846F0
S1131090FFF770FF38BD2846FFF7B4FF38BD284678
S11310A0FFF78CFF38BD42F2797038BD42F27B7095
S11310B038BD00BF08B50F4B0F4A5A62DB684BB10D
S11310C00C4A1269934211D90A4801320261036839
S11310D0984708BD074B9B6E1BB9064803689847A1
S11310E008BD013B034A9366002008BD42F27470B8
S11310F008BD00BFF404FF1FE004FF1F2DE9F843FF
S1131100074688460024A446124DA14619E02B69DF
S1131110C3F11003C4EB080207E02E69711C2961B6
S1131120395DA955013B013A01340BB1002AF4D1D0
S113113033B9C5F81090FFF7BDFF844608B105E048
S113114012B14445E3D101E042F27D7C6046BDE842
S1131150F88300BFE004FF1F10B50B4B93F8593020
S1131160042B0BD1084BDC6D54B1002004F0CCFAF5
S1131170054B586EA04742F27E7010BD002010BD92
S113118042F27E7010BD00BFF404FF1F184B9B6831
S11311901B69013817281FD8DFE800F00C0C0C0C71
S11311A00C0C0C0C1E0F0C0C140C0C0C0C1E1E1E28
S11311B01E191E0C42F63D00704701290FD8196311
S11311C00020704701290DD8596300207047022977
S11311D00BD899650020704742F63C00704742F6F0
S11311E03E00704742F63E00704742F63E007047AC
S11311F01004FF1F38B50C4B9B681C6904F1700583
S1131200284648F2C031302204F0F6FD226F074B25
S11312109A4204D02846FF21302204F0F6FD04F05F
S11312209BFC002038BD00BF1004FF1F6B63666782
S11312302DE9F047DFF83C81D8F808301C694B23CE
S1131240E3700126A6704FF0050984F8019026701A
S11312505023E371A6714FF0020A84F805A0002719
S113126027715423E372A67267722772266366633A
S11312704EF6FF73A36308F120052846042104F108
S1131280100201F09BFE2846314604F1140201F0DD
S113129095FE2846394604F1180201F08FFE2846CF
S11312A0514604F11C0201F089FE2846032104F191
S11312B0200201F083FE2846494604F14C0201F065
S11312C07DFE2846062104F1500201F077FE2846EF
S11312D0072104F1540201F071FEA3695B42204A24
S11312E01A40204961EA0303226663661E4BA36623
S11312F01E4BE366D8F81400E760394607E094F81B
S11313008020134202D0E2681343E360013101EB11
S11313104103DB00C358002BF1D1154B41F25402B9
S11313209A58A26441F258029A58626441F25C02EB
S11313309A58226403F583531B68E3630D4B5B687F
S1131340DA6862621A69DB68D31A0133A362204641
S113135003F0E0F80123A3650020BDE8F08700BF97
S113136000000000B36100000000FF1F0000032024
S1131370007004401004FF1F30B583B014461D46AE
S11313803A4B9B681B690138172869D8DFE800F0DD
S11313900C0E1114171A232668292F382C1D203BF4
S11313A0435154575A5D6860042253E00C330422BD
S11313B050E0103304224DE0143304224AE0183381
S11313C0042247E02033042244E02433042241E091
S11313D0283304223EE0383304223BE02C33042239
S11313E038E03033042235E03433042232E01F4B3A
S11313F0D86943695B6998471D4B1860042229E04A
S11314006033102226E041F224031A4AD258184BC2
S11314101A6004221EE018480DF1070101F002FED3
S11314209DF80720003218BF0122114B1A600422D4
S113143010E03C3310220DE04C3304220AE0503318
S1131440042207E05433042204E05833042201E068
S11314500833042205B12A602CB12360002003E084
S113146042F63C0000E0002003B030BD1004FF1F32
S11314706405FF1F007004403004FF1F074BD3F8BE
S11314808820511CC3F888101A4482F82000D3F82D
S1131490882002F03F02C3F8882070472006FF1F0F
S11314A000207047034B012283F89220002283F826
S11314B0902070472006FF1F2020704738B505464E
S11314C00A46034BD869046964682946A04738BDB5
S11314D01004FF1F2DE9F84F83468A46144600F096
S11314E0A3FF06460F464FF47A7000FB04F000F0A9
S11314F0B5FF044600254FF00009DFF8588021E0CD
S113150054EA050308D000F08FFF801B61EB07014C
S1131510A94208BFA0421AD2D8F88C30D8F8882043
S113152093420FD05A1CC8F88C20434493F82030BF
S11315300BF80930D8F88C3003F03F03C8F88C302E
S113154009F10109D145DBD10020BDE8F88F052060
S1131550BDE8F88F2006FF1F70B50446012600255C
S1131560204631462A46FFF7B5FF18B923785A2B8F
S1131570F6D170BD70BD00BF10B50446FFF7ECFF97
S113158028B9601C01210A22FFF7A4FF10BD10BD79
S113159030B583B0134C04F1600501A8FFF7ECFFEC
S11315A0B8B99DF8053003F15F02D2B2022A11D80E
S11315B0A32B11D0A22B06D1B4F862102846063111
S11315C0FFF77CFF58B99DF80530A22BE5D0002029
S11315D005E004E0042002E042F21270FFE703B0E9
S11315E030BD00BF2006FF1F10B582B0044601A81D
S11315F002211422FFF76EFFBDF80430638002B0AD
S113160010BD00BF10B582B0044601A80221142207
S1131610FFF760FFBDF80430A38002B010BD00BF27
S113162030B583B004460D4601A802F0ADFE01A812
S11316302146042202F0ACFE01A82946628802F089
S1131640A7FE01A80DF1060102F0BEFEBDF80600DA
S113165003B030BD00B583B05A238DF804308DF843
S113166005000122044B83F8912001A80221FFF711
S113167025FF03B05DF804FB2006FF1F08B50D4BE2
S113168093F890303BB100220A4B83F89020A120BC
S1131690FFF7E0FF08BD074B93F892303BB10022FF
S11316A0044B83F89220A320FFF7D4FF08BD002049
S11316B008BD00BF2006FF1F08B5FFF7DFFF08BD08
S11316C070B5A0B014461D460E46002938D0202A15
S11316D038D8FFF7D3FF002836D11D4B93F891304B
S11316E01BB100221A4B83F89120194B5A2283F81C
S11316F06020A42283F8612015B1A52283F861201B
S1131700134BA3F8624054B103F1660031462246FC
S113171004F072FB68463146224604F06DFB0C4E21
S113172006F1600528466946FFF77AFFA6F86400CB
S11317302846A11DFFF7C2FE38B9FFF729FF04E0D0
S1131740042002E0042000E0FFE720B070BD00BFE9
S11317502006FF1F10B582B00446104B93F890305A
S11317603BB10E4B93F891301BB10C4B93F8923074
S11317707BB90B4B1B88ADF8043023695B682046AA
S113178001A90222984723695B682046054908227B
S1131790984742F2137002B010BD00BF2006FF1F2D
S11317A01C5E00003C5E000070B504460E46154603
S11317B0FFF7E2FE58BB6378A62B04D1164BD86919
S11317C0FFF7C8FF70BD0DB9A42200E0A5229A421C
S11317D01ED12046FFF708FFE0B96388202B28BFFD
S11317E0202363802046FFF70DFF034698B96288E3
S11317F05AB13046002104F008FB618801EB8102F4
S113180052003046FFF766FE0346184670BD70BDB1
S1131810012070BD70BD70BD1004FF1F2DE9F0479D
S1131820A2B091461F468A46002941D0002A41D0E1
S113183000231360224A82F89130FFF71FFF00282B
S11318403AD11F4D00264FF0200828463146424623
S113185004F0DBFA20A829463A46FFF7A5FF18B1A1
S11318600022C9F8002027E0BDF882201AB168469A
S1131870294604F0C1FA20A86946FFF7D1FEBDF855
S11318808430834201D1012400E0344614B9A220FB
S1131890FFF7E0FE002CD8D0094B012283F89020FA
S11318A0CAF80030BDF88230C9F80030002003E0E7
S11318B0042001E00420FFE722B0BDE8F08700BF68
S11318C02006FF1F30B420E010F0010F01D10129E0
S11318D005D112F8013B00F8013B013915E010F085
S11318E0020F01D1032904D832F8023B20F8023B4D
S11318F002398D0809D0AD00441903E052F8043BC5
S113190040F8043BA042F9D3491B0029DCD130BC88
S1131910704700BF08B5034610461A46FFF7D2FFCA
S1131920002008BD08B5FFF7CDFF002008BD00BFAB
S113193008B50B4611461A460123FEF705FE08BDFD
S113194030B583B00A4D6C68203528460421224600
S113195001F034FB2846012101AA01F02FFB226883
S1131960019B1344013B6360002003B030BD00BF02
S11319701004FF1F08B500F091FA08BD2DE9F043EB
S113198089B08046174621F00706324B9C682469CB
S1131990D4F830904FF0FF344FF0FF35CDE90645D1
S11319A011F0070504D006A891192A4604F024FA78
S11319B0FFF76CF93EB1284841463A46334601F0F8
S11319C0D9FB044600E0002444B93DB1224808EBA9
S11319D0060106AA082301F0CDFB0446FFF75EF9D1
S11319E0002C31D1B9F1000F30D0FFF74FF986B197
S11319F0184883681B6993F85830009304AB01932B
S1131A0005AB02932030414632463B4601F03CFD93
S1131A10044694B98DB10F4883681B6993F8583014
S1131A20009304AB019305AB0293203008EB06014D
S1131A30082206AB01F028FD0446FFF72FF90CB18C
S1131A40204604E0002002E0204600E0002009B027
S1131A50BDE8F0831004FF1F3004FF1F2DE9F04F91
S1131A608DB004468B464A4B9B681B691B6B13F174
S1131A70000818BF4FF0010810460021CDE9040109
S1131A8011460020DDE90423801841EB0301CDE970
S1131A900A010BF00703042B07D9CBF1000525F04D
S1131AA007056D424FF0000B2FE02BF00705C5EB47
S1131AB00B0B2AE0FFF7EAF8384621460AAA082366
S1131AC001F058FB0646FFF7E9F8002E5AD1B8F1A9
S1131AD0000F17D0FFF7DAF8D9F808301B6993F82C
S1131AE05830009307AB019308AB0293504621464C
S1131AF008220AAB01F0C8FC0646FFF7CFF80EB186
S1131B00304642E00834083D04E0224FA7F12009A2
S1131B1009F1200A002DCDD1BBF1000F34D0DDE94D
S1131B200401003041F1FF310CAD65E90401FFF718
S1131B30ADF8184821462A46082301F01BFB064647
S1131B40FFF7ACF8E6B9B8F1000F17D0FFF79EF82D
S1131B500F4883681B6993F85830009306AB0193D0
S1131B6007AB029320302146082208AB01F08CFC1D
S1131B700446FFF793F80CB1204606E0002004E089
S1131B80304602E0304600E000200DB0BDE8F08FA2
S1131B901004FF1F3004FF1F70B506460D46FFF703
S1131BA075F8104831462A460F4B01F0ABF904464C
S1131BB0FFF774F89CB90D4B9B681B691B6B73B1E1
S1131BC0FFF764F8094883681B69203031462A46C8
S1131BD093F8583001F002FC0446FFF75FF8204602
S1131BE070BD00BF3004FF1F6B66656B1004FF1FE0
S1131BF038B5274B9B681C69236E1BB9626E1AB1FA
S1131C00002202E0002200E001221146A569626B75
S1131C10EAB1E1B933B16942194005D00020FFF7B8
S1131C20BBFF02E0002000E0002000282FD1184B69
S1131C305968626E52426D4215406B424A689A423C
S1131C4025D9A91818460131FFF7A6FF38BDFFF7BB
S1131C501DF81048104901F099F90446FFF71EF8E1
S1131C6094B90B4B9B681B691B6B6BB1FFF70EF8A8
S1131C70074883681B69203093F8581001F0F4FB7F
S1131C800446FFF70BF80CB9204638BD204638BD92
S1131C901004FF1F3004FF1F6B66656B08B5074B0C
S1131CA01B6833B11B6933B198470022034B1A6098
S1131CB008BD002008BD002008BD00BFB406FF1FFA
S1131CC030B4164B5B68136013E01C681CB95D6884
S1131CD00DB99D68ADB1844209D85C68844206D3CD
S1131CE04318013B9C420FD242F2D87013E00C33EC
S1131CF0136059B16AB11368002BE6D142F2D8706F
S1131D0009E042F2D87006E0002004E042F2D87004
S1131D1001E042F2D87030BC704700BF1004FF1FCE
S1131D2070B582B0054616460C4671B101AAFFF79C
S1131D30C7FF034638B9019B9B685B682846214668
S1131D40324698470346184600E0002002B070BDB2
S1131D5010B5064B5C6803E01B6803B198470C346C
S1131D60A368002BF8D1002010BD00BF1004FF1F92
S1131D7070B4104B9B681A69536BB3B101440139B9
S1131D8000230EE003F10C0402EBC40552F83440C6
S1131D900CB96E6826B16D68854201D3A14206D2A2
S1131DA00133012BEEDD002002E0002000E00120E1
S1131DB070BC70471004FF1F70B582B0054616460C
S1131DC00C46E1B1FFF7D4FFD8B92846214601AA51
S1131DD0FFF776FF034680B9019B9B689B68284602
S1131DE0214632469847034620B9019A9168074A2A
S1131DF0116002E00021054A1160184603E000204A
S1131E0001E042F2D87002B070BD00BFB406FF1FFB
S1131E1070B582B005460C4601AAFFF751FF034690
S1131E2068B9019B9B685E6966B128462146FFF745
S1131E309FFF48B928462146B047034600E034B125
S1131E40184605E0662003E042F2D87000E0002066
S1131E5002B070BD70B582B0054616460C4699B105
S1131E60FFF786FF90B92846214601AAFFF728FF0D
S1131E70034638B9019B9B68DB68284621463246F5
S1131E8098470346184603E0002001E042F2D87068
S1131E9002B070BD08B500F035F808BD10B50446B1
S1131EA00B46104621461A4603F0A6FF002010BD3B
S1131EB070B50B46144610F0030F15D0B0F1005F57
S1131EC012D24218013AB2F1005F0DD3C0F10055AD
S1131ED04E1B21462A4603F08FFF4FF00050611934
S1131EE0324603F089FF03E021461A4603F084FFDB
S1131EF0002070BD08B50B4611461A460123FEF7B3
S1131F0023FB08BD214B1B68C3F30333033B082B9E
S1131F101BD8DFE803F0051C080B0E11141A170078
S1131F204FF4804315E04FF4004312E04FF4404374
S1131F300FE04FF480330CE04FF4C03309E04FF46A
S1131F40003306E04FF4802303E0002301E04FF464
S1131F50C043CBB123B15A1E134203D1012202E084
S1131F60012200E000220AB1032200E00222084913
S1131F704968501CB3FBF0F3C3F10050C8606FF024
S1131F80604002FB03030B610020704700700440B3
S1131F901004FF1F0023C370837003700422427077
S1131FA083724374704700BF2DE9F003604C2360D3
S1131FB04FEA021891FBF8F84FEA0813B1FBF3F368
S1131FC014469A4201D908F1FF38934214D14FF0D4
S1131FD0000C4FF0FF351AE09946F118B7FBF1F108
S1131FE08C4201D2091B00E0611AA94201D8CC46F7
S1131FF00D460133DBB208E04FF0000C4FF0FF3523
S1132000012301FA03F74FEA4816202BE4D9494B80
S113201083FB0213D217C2EB631202EB4202AA4201
S113202040F28180444B98422CD008D8A3F5005349
S1132030984210D003F58053984218D04DE03F4B9E
S1132040984235D003F5805398423CD0A3F5FC2345
S1132050984242D121E04FF00042394B1A60394A8C
S113206041F23403D15841F48061D15035E0022269
S1132070334B5A60334A41F23403D15841F400617E
S1132080D1502AE008222E4B5A602E4A41F23403E2
S1132090D15841F48051D1501FE02022284B5A607E
S11320A0284A41F23403D15841F40051D15014E08C
S11320B00422234B9A60234A41F22803D15841F465
S11320C08061D15009E010221D4B9A601D4A41F2F3
S11320D02803D15841F40061D150C37803F0F303CD
S11320E0C37000238370027802F0E002C8F3042175
S11320F00A4302705FFA88F880F80180827A02F05D
S1132100E00242EA0C0C5FFA8CFC80F80AC0C022A0
S11321104274C27842F02002C270C27842F00C02CB
S1132120C270184600E00120BDE8F003704700BF0C
S1132130B806FF1F1F85EB5100C0064000A00E40EB
S113214000E100E000700440037913F0800FFBD03D
S1132150C9B2C171704700BF08B5054B1B7913F0B4
S1132160200F04D0024BD879024B1B68984708BD56
S113217000A00640B806FF1F08B5094B1B79DBB267
S113218013F0020F02D0064BDB7908BD13F0200FC9
S113219004D0034BD879034B1B68984708BD00BF94
S11321A000B00640B806FF1F08B5054B1B7913F0B5
S11321B0200F04D0024BD879024B1B68984708BD06
S11321C000C00640B806FF1F08B5054B1B7913F085
S11321D0200F04D0024BD879024B1B68984708BDE6
S11321E000D00640B806FF1F08B5054B1B7913F055
S11321F0200F04D0024BD879024B1B68984708BDC6
S113220000A00E40B806FF1F08B5054B1B7913F05C
S1132210200F04D0024BD879024B1B68984708BDA5
S113222000B00E40B806FF1F10B50446564B984246
S11322302ED008D8A3F50053984210D003F580534C
S1132240984219D053E0514B984239D003F580534A
S1132250984241D0A3F5FC23984248D124E04FF0A2
S113226000424B4BC3F880204A4A41F23403D15810
S113227041F48061D1503AE00222454BC3F88420F6
S1132280444A41F23403D15841F40061D1502EE064
S113229008223F4BC3F884203E4A41F23403D1580C
S11322A041F48051D15022E02022394BC3F88420DC
S11322B0384A41F23403D15841F40051D15016E068
S11322C00422334BC3F88820324A41F22803D15800
S11322D041F48061D1500AE010222D4BC3F88820CC
S11322E02C4A41F22803D15841F40061D1502046D0
S11322F0FFF750FE244B9C4225D008D8A3F5005389
S11323009C4210D003F580539C4214D010BD1F4B47
S11323109C4228D003F580539C422CD0A3F5FC2387
S11323209C422FD117E01B4A41F23403D15821F4C7
S11323308061D15010BD174A41F23403D15821F4C1
S11323400061D15010BD134A41F23403D15821F435
S11323508051D15010BD0F4A41F23403D15821F4B9
S11323600051D15010BD0B4A41F22803D15821F439
S11323708061D15010BD074A41F22803D15821F49D
S11323800061D15010BD00BF00C0064000A00E4047
S113239000E100E0007004400C4BDB7803F07F03A5
S11323A0042B11D1094B5A7802F09F025A70002372
S11323B00649074806E0CA7802F07F02012A00D1E4
S11323C082780133FE2BF6DD704700BF00E0074042
S11323D000D0074000220B4B1A600B4B6FF07F417B
S11323E059609A6007221A60084B1B68DB00084A90
S11323F0A2FB03139B0C074A136013B90122054B7C
S11324001A607047BC06FF1F10E000E00004FF1FC5
S113241083DE1B43C006FF1F024B1A6822F006022C
S11324201A60704710E000E030B40A4B0A491C6897
S11324308A68D24322F07F401A689442F7D100237D
S113244043EA14232206141843F1000520462946C2
S113245030BC7047BC06FF1F10E000E0024B1B6855
S113246003FB00F0C0087047C006FF1F014B18684B
S1132470704700BF0004FF1F024B1A6801321A6044
S1132480704700BFBC06FF1F10B5274B53F8203020
S1132490DA7802F0ED0242F00202DA70234A52F8CE
S11324A020009A78C2F30011DA7812F0200F3AD0A3
S11324B09A7812F0200F36D091B1DA7812F0010F29
S11324C003D00522027401220DE0C268013AC26001
S11324D042B18268541C846052781A71002202E06E
S11324E0002200E00122D1B941680139416011B1F3
S11324F0012906D00AE09A7802F0CF029A700122EC
S113250008E0997841F00801997003E0997801F0A6
S1132510F701997001684C1C04601B790B7012B1AF
S11325201830FEF79BFB10BDC05E0000C406FF1F01
S113253008B50020FFF7A8FF08BD00BF08B50120BB
S1132540FFF7A2FF08BD00BF08B50220FFF79CFFFC
S113255008BD00BF08B5034B53F8200000F07AFB18
S113256008BD00BFD05E000008B5044B53F820003E
S1132570114600F0E5FB002008BD00BFD05E00005E
S113258010B5084C54F8200021B911461A4600F041
S1132590B3FB10BD012903D111461A4600F0C0FB5C
S11325A010BD00BFD05E00002DE9F8430446894603
S11325B090461E46089B2F4A52F8205000EB4002DA
S11325C092002D4F174493E8070087E807002B4A31
S11325D041F23C03D15841F01001D15028469DF8F6
S11325E0241000F0F7F9284600F0D8F9284600F046
S11325F01DFB2846D9F8001000F054FB28460021A2
S113260000F0AEFB06F110000021FEF7CFFA06F150
S113261028000021FEF7CAFA194B1B5D5AB2520971
S113262003F01F03012101FA03F0164B43F82200C3
S1132630154A125D50B2400902F01F0201FA02F27B
S113264043F82020114A125D50B2400902F01F02E3
S1132650914043F82010B8F1000F02D0284600F052
S1132660C5FA002333607360094B43F82460BDE866
S1132670F88300BFD05E0000D006FF1F0070044046
S1132680D45E000000E100E0CC5E0000D85E0000F3
S1132690E806FF1F70B586B00B4D55F820500B4E61
S11326A056F8200081605468059412788DF8102043
S11326B006AA082042F80C0D00200090284600F0DD
S11326C0A9F906B070BD00BFD05E0000E806FF1F88
S11326D02DE9F04387B088460F9D164C54F82060CE
S11326E0154C54F820705068059012788DF810201D
S11326F006AA0C2042F80C0D0E980090384600F003
S113270089F9814690B93846414600F05FFA10369F
S113271030462946FEF768FA04460328F8D03846BE
S1132720414600F05BFA0CB14FF00509484607B08A
S1132730BDE8F083E806FF1FD05E0000F0B585B069
S11327400C461E46154D55F82050154F57F82000DD
S113275041605068039012788DF8082004AA0F2075
S113276042F80C0D284600F0BFF998B904AA0023DA
S113277042F80C3D28462146334600F0B5F950B9DD
S113278004AA042342F80C3D28462146334600F0AF
S1132790ABF900E0FFE705B0F0BD00BFD05E00007C
S11327A0E806FF1F38B50446284B53F8205041F281
S11327B03C03274AD35813F0100F44D005F11000FE
S11327C0FEF75AFA05F12800FEF756FA214B1B5D75
S11327D059B2490903F01F03012202FA03F01E4B08
S11327E0203143F821001D49095D48B2400901F038
S11327F01F0102FA01F1203043F820101849095D45
S113280048B2400901F01F0102FA01F1203043F8F7
S113281020101449095D48B2400901F01F018A40A3
S1132820203043F82020104B53F8240000F0E6F841
S11328300022064B43F82420054A41F23C03D158B8
S113284021F01001D150002038BD00BFE806FF1F61
S113285000700440DC5E000000E100E0D45E000093
S1132860CC5E0000D85E0000D05E00002DE9F0418F
S113287086B00446264B53F82050264B53F820705C
S113288000EB40039B00244A02EB03082A6BAB6A6B
S11328901A400592059A002A33D07B68012202FA75
S11328A003F3059A1A421FD007F12800FEF7D6F960
S11328B07968284600F086F9796828466A4600F067
S11328C047F958B10FE006AA3244D8F8043012F898
S11328D00F0C214698470136F6B200E000269DF819
S11328E00830B342EFD8AB68BB68012202FA03F3A5
S11328F0059A1A4203D007F11000FEF7AFF9059BC1
S11329002B63284600F0F0F906B0BDE8F08100BF63
S1132910D05E0000E806FF1FD006FF1F08B5034B7A
S113292053F8200000F052F908BD00BFD05E00004B
S113293008B5034B53F8200000F012FA08BD00BF9D
S1132940D05E000008B5034B53F8200000F064FA91
S113295008BD00BFD05E000000EB40008000024BC9
S113296018444160704700BFD006FF1F08B500201F
S1132970FFF77CFF08BD00BF08B5002002F0EAFDA8
S113298008BD00BF08B5002002F0EEFD08BD00BF81
S113299008B50020FFF76AFF08BD00BF036813F401
S11329A0801F07D0036823F000430360036813F417
S11329B0801FFBD1704700BF0368002B08DB00F1C8
S11329C004735B010122DA67036813F4801FFBD0F0
S11329D0704700BF00F10470043040014163704748
S11329E0036813F4801F08D100F104735B01012212
S11329F05A66036813F0007FFBD1704738B504466C
S1132A00FFF7EEFF002565602046FFF7D5FF656000
S1132A1038BD00BF2DE9F0018846059911B300EBDC
S1132A2008150024C5F88840C5F88C402F4616E0E8
S1132A300D5D032C09D86642F6001836B540D7F868
S1132A4088603543C7F8885008E06642F600383697
S1132A50B540D7F88C603543C7F88C50013495687D
S1132A60A542E5D808F1080109014418656825F074
S1132A70FF5525F4E015656065681A4E06EA834340
S1132A802B436360435823F4C0034350435823F457
S1132A90702343504458936844EA034343501368F3
S1132AA00F2B1BD01C2B06D10B46415841F480112F
S1132AB0C1500C23136008F108084FEA081850F8B5
S1132AC0083023F0706340F8083050F80810136899
S1132AD01B0603F070630B4340F808300020BDE888
S1132AE0F00170470000FC1FF0B401F10804240158
S1132AF00519065926F4C0060651065926F470260F
S1132B0006510759966847EA064606516C6824F050
S1132B10FF5424F4E0146C606C680C4E06EA8343A2
S1132B201C436C6013680F2B0CD008310901435807
S1132B3023F070634350445813681B0603F070631A
S1132B40234343500020F0BC704700BF0000FC1F2B
S1132B5070B401F108031B01C358136013F4001F80
S1132B6009D001F1080300EB03135B6853600023F1
S1132B7000EB01151BE001F1080300EB03135B6894
S1132B809B0C5360F3E7032B06D8D5F88860DC0070
S1132B90E640D41A267309E0D5F88C6003F100549A
S1132BA0043CE40026FA04F4D61A34750133072BE6
S1132BB0E9D90831090143581B0C1372002070BC79
S1132BC0704700BF0831090143587047836A0122E6
S1132BD002FA01F10B438362704700BF836A01224A
S1132BE002FA01F123EA01038362704700F10470E1
S1132BF00430400101238363704700BF00F1047374
S1132C005B0100221A679A67036813F0807FFBD187
S1132C10704700BF00F104735B0101229A671A67D1
S1132C20036813F0807FFBD0704700BF10B50446E3
S1132C30FFF7D6FE2046FFF7EDFF054B23616361E6
S1132C40A3612046FFF7DAFF0023A36210BD00BF93
S1132C50FFFF030038B504460D46FFF7DBFF63684A
S1132C6023F007031B041B0C63606268297801F0DE
S1132C700701AB781B0403F4E0230B436978C90410
S1132C8001F460110B43E97843EA0163297989056A
S1132C9001F440010B43134363602046FFF7AEFF8A
S1132CA038BD00BF70B504460E46FFF7B3FF226877
S1132CB022F07F0206F07F031343236000231A46A9
S1132CC00CE003F108000001251822506A6004EBAF
S1132CD00310C0F88820C0F88C200133B342F0D32D
S1132CE02046FFF78BFF70BD036A13F0070F01D076
S1132CF007230362704700BF70B504460D461646AD
S1132D00FFF788FF054B03EA864605F5087544F886
S1132D1025602046FFF772FF70BD00BF0000FC1F56
S1132D2070B504460D461646FFF774FFC6F3110648
S1132D3005F5087544F825602046FFF75FFF70BD70
S1132D4038B504460D46FFF765FF044B03EA854595
S1132D5025612046FFF752FF38BD00BF0000FC1F6D
S1132D6038B505460C46032902D1FFF753FF06E0A8
S1132D70042904D100F104735B010122DA672846B7
S1132D80FFF748FF2CB905F104735B010022DA65F3
S1132D9010E0012C06D105F1047304335B01012218
S1132DA0DA6007E0022C05D105F1047304335B01FA
S1132DB001221A632846FFF721FF38BD38B50546BE
S1132DC00C46032902D1FFF719FF05E0042903D1BA
S1132DD0036823F0004303602846FFF71BFF2CB968
S1132DE005F104735B010122DA6510E0012C06D1C0
S1132DF005F1047304335B010022DA6007E0022C5E
S1132E0005D105F1047304335B0100221A632846DB
S1132E10FFF7F4FE38BD00BF036843F0007303609E
S1132E20036813F0007FFBD1704700BF036843F4CD
S1132E3070030360BFF36F8FBFF34F8F704700BF02
S1132E40704700BF10B50446044B591E044AD21AF9
S1132E5002F0D2FF0134034B1C6010BD2D2E000084
S1132E60412E0000EC06FF1F08B500F0F9F818B970
S1132E70024B1B680248984708BD00BFEC06FF1FC1
S1132E8004F0014080230370037813F0800FFBD01B
S1132E90704700BF704700BF10B50446044B591E6D
S1132EA0044AD21A02F0A8FF0134034B1C6010BD7F
S1132EB0852E0000952E0000F006FF1F10B570222D
S1132EC00E4B1A7000F0CCF888B90C4C0C4B1B68F4
S1132ED0204698472378DBB213F0200F08D113F073
S1132EE0100F07D113F0010F06D0692010BD10BDDB
S1132EF0672010BD682010BD002010BD00000240F6
S1132F00F006FF1F2DE9F84F05460C461746984674
S1132F10102300F0F3F8064678BB2744013FEB6822
S1132F20B7FBF3F203FB1272CAB1B7FBF3F707FB6B
S1132F3003335F1E13E0DBF800301C608AF807904F
S1132F40404600F0F9F8D0B92846FFF7B7FF064627
S1132F502B6903B1984756B9EB681C4405E0DFF8C8
S1132F6024B0DFF824A04FF00909BC42E3D9284675
S1132F70FFF77AFF3046BDE8F88FBDE8F88FBDE86B
S1132F80F88F00BF005F00000000024038B504461F
S1132F9078B14422084BDA71084600F0CDF850B9F4
S1132FA02046FFF78BFF05462046FFF75DFF2846C6
S1132FB038BD042038BD38BD000002400346002857
S1132FC029D0002A29D0072929D8DFE801F00408EC
S1132FD00C1115191C20DB681360002070475B6816
S1132FE01360002070475B685B0813600020704723
S1132FF09B681360002070471B68136000207047B3
S11330000020106070475B691360002070479B6963
S113301013600020704704207047042070476A2022
S1133020704700BFB0B1B9B10C4B9B78DBB203F071
S11330300302022A02D100200870704703F0C00383
S1133040802B03D101230B700020704702230B70E7
S1133050002070470420704704207047000002409D
S113306030B1C36933B11B68022B05D06D207047A2
S1133070042070476D2070470020704710B550B190
S1133080C4696068FFF708FFA068FFF7DBFE02234E
S11330902360002010BD042010BD00BF10B50446FD
S11330A000B341F24C03124AD258C2F30362114BEB
S11330B033F812301A03BBB10023036042600222CA
S11330C082604FF48052C260436183610361FFF701
S11330D0C7FF034648B1084BE3612046FFF7CEFF24
S11330E0002302E0042300E06423184610BD00BF5F
S11330F000700440E05E00000404FF1F10B470B1CF
S1133100013B0B420DD113420DD103688B420CD805
S11331100A4441680B449A4209D9662008E0042015
S113312006E0652004E0652002E0662000E000205F
S11331305DF8044B704700BF034B984201D06B20ED
S113314070470020704700BF6B66656B50B112B1C9
S1133150082A03D008E049B1042070470B2907D995
S113316004207047042070470420704700207047F3
S1133170002070472DE9F84F80460E461D4617463D
S11331806AB31A460823FFF7B9FF8146D8B129E08C
S1133190DBF800301E603C4654F8082B5A607A680D
S11331A09A60114B83F807A04046FFF787FE8146DB
S11331B0D8F8103003B19847B9F1000F09D1083697
S11331C0083D274603E0DFF824B04FF0070A002D3E
S11331D0DED14046FFF748FE4846BDE8F88F04209C
S11331E0BDE8F88FBDE8F88F00000240005F0000E2
S11331F0F8B504460D461E461746DAB11A46FFF7DF
S1133200A5FFC8B90D4B4322DA71EAB29A710C4B8F
S11332101B683A685A600B2D03D8082E01D17A68CE
S11332209A602046FFF74AFE05462046FFF71CFE3B
S11332302846F8BD0420F8BDF8BD00BF00000240D8
S1133240005F0000F8B505460C461E461746CAB195
S11332501A46FFF77BFFB8B90C4B4122DA71E2B290
S11332609A712846FFF72AFE034648B9084A1268AD
S1133270516839600B2C03D8082E01D192687A600A
S11332801846F8BD0420F8BDF8BD00BF0000024098
S1133290005F000010F0070F20D111F0070F1FD1BD
S11332A0012A1FD8014401F1FF3305D108281BD19D
S11332B010291BD100207047D2B9B3F5806F19D300
S11332C0B0F5802F02D30F4A934215D9B0F5002FE1
S11332D014D30D4A934213D90420704765207047D4
S11332E0652070470420704704207047042070470D
S11332F0002070470020704700207047042070476A
S113330000207047FF030400FF0308002DE9F84F75
S11333100F4616461D469DF82890824638B34AB398
S1133320084619464A46FFF7B5FF0146B0B124E006
S1133330134B1C68276088F807B088F80B90504638
S1133340FFF7BCFD014678B96268334643F8082BA1
S1133350A26872600837083D1E4603E0DFF8248047
S11333604FF0030B002DE3D10846BDE8F88F04208D
S1133370BDE8F88F0420BDE8F88FBDE8F88F00BFE2
S1133380005F00000000024008B50246F8B101B336
S1133390114B9B7803F00303022B16D00E4B4520F0
S11333A0D8710878D8724878987288785872C87832
S11333B018720879D8734879987388795873C979D9
S11333C019731046FFF77AFD08BD002008BD0420DC
S11333D008BD042008BD00BF000002402DE9F04FE5
S11333E083B081460E46154601931023FFF786FEEF
S11333F090BBD9F80420D9F80830B2FBF3FA734231
S1133400CAF100021340C3F10008B0451DD1C3EB5B
S11334100A081AE0C6EB0804AC4200D92C46DBF8D3
S113342000301E604FF00103FB71C4F30733FB72DD
S1133430C4F30713BB72019B7B724846FFF73EFD42
S113344058B92D1B2644D04402E0DFF818B0044FCD
S1133450002DDFD1002000E0FFE703B0BDE8F08FCE
S113346000000240005F000008B5024638B1054B79
S11334704020D87199711046FFF720FD08BD042043
S113348008BD00BF000002402DE9F84F80460D46FC
S113349014469DF828901E4653B30423FFF72EFECE
S11334A00346D8B127E0DBF800301D6087F807A099
S11334B087F80B9032689A604046FFF7FFFC03469A
S11334C040B10B9901B10D600C9A72B100220C99B4
S11334D00A600AE0043C0436043504E0DFF820B056
S11334E0064F4FF0020A002CDDD11846BDE8F88FD4
S11334F00420BDE8F88FBDE8F88F00BF000002404B
S1133500005F000008B5002000F094FA08BD00BF79
S113351008B5012000F08EFA08BD00BF08B50220EE
S113352000F088FA08BD00BF2DE9F04F85B0574B75
S113353053F82060564B53F82070337A8DF80A30D4
S113354033788DF80930737A8DF8083000238DF8BC
S11335500B308DF80C30384602A900F035FE824657
S1133560F369D6F820B07268082A38D84FF00008FA
S1133570484D494C7EE0F369022B17D18DF80B803E
S11335808DF80850384602A900F01EFE8246736981
S1133590BBB196F840200AB11C7812E01A4612F822
S11335A0011B72615C7841EA04240AE0726942B149
S11335B0134613F8011B7361547841EA0424013360
S11335C0736144EA0A037B634FF00073FB62F3699F
S11335D0023BF361F369002B54D0F36903E0002448
S11335E04FF001082546FA6A12F0007F4AD0C3EB77
S11335F00B03072BBFD945E0F369012B0BD14FF027
S113360001008DF80B0004A9002301F8083D384699
S113361000F0DAFD8246736913B113F8018B73610C
S113362095F8009009F1FF3303F02F0304EBC30373
S1133630D3E90001CDE9000109F101032B70FEF784
S1133640F3FEDDE90023801A61EB030104EBC909F1
S1133650C9E900012B7803F03F032B7048EA0A0301
S11336607B634FF00073FB62F369013BF361F36921
S113367043B1F369FA6A12F0007F03D0C3EB0B0382
S1133680032BB9D905B0BDE8F08F00BF3407FF1F85
S1133690045F00004007FF1F4807FF1F70B50E4B73
S11336A053F820600D4B53F8205000246C6334749D
S11336B028462146224600F069FD28462146224636
S11336C000F052FD96F8243013F0FF0F03D006F1FA
S11336D02800FDF7C3FA70BD3407FF1F045F000024
S11336E0F0B583B007460D461646374B53F82040D5
S11336F008460021482202F088FB012F0BD017B1A5
S1133700022F10D05DE0314A41F23C03D15841F41C
S11337108051D1500EE02D4A41F23C03D15841F47E
S11337200051D15006E0294A41F23003D15841F406
S11337308051D15002F07EF9E86033782B70F37831
S11337402B72B3786B72204600F0F2FB05F128006F
S11337500021FDF72BFA236843F0004323607378BC
S1133760226822F080429B0703F0804313432360C6
S11337702046F178327900F093FB204601210A4675
S113378000F0A0FB31780126009620460022334643
S113379000F04CFC0E4B43F827500E4BDB5D59B246
S11337A0490903F01F039E400B4A42F82160236835
S11337B023F480432360236823F001032360002063
S11337C000E0072003B0F0BD045F00000070044077
S11337D03407FF1F105F000000E100E0F0B583B084
S11337E00F4614461E460A4B53F82050094B53F813
S11337F020002978EB6800923A4600F05DFC3060C6
S1133800844201D8002000E0082003B0F0BD00BFCE
S11338103407FF1F045F00002DE9F0410E46904677
S11338200C4B53F820400C4B53F820700D4638468F
S1133830217855F8042BE36800F0C0FAC8F80000BA
S1133840384621782A4600F091FB73686360BDE82E
S1133850F08100BF3407FF1F045F0000F0B583B0A0
S113386006460F46294B53F82050294B53F8204065
S11338702B7C13F0FF0F46D121B101AAFFF7CCFF37
S11338807B686B606B68082B0DD9EB6913F0010F33
S113389009D0EB690133EB612B6A01332B620123FD
S11338A085F8403002E0002385F8403001272F746A
S11338B023683B432360204639463A4600F026FB02
S11338C04FF00043E3624FF08053E3624FF0006334
S11338D0E3624FF00073E3624FF40023E3624FF4BA
S11338E00033E362A3689BB2A360236823F001035F
S11338F023603046FFF718FE204600213A4600F0C8
S113390045FC002000E0042003B0F0BD3407FF1F95
S1133910045F000008B5064B53F820301B7C13F0FD
S1133920FF0F03D0FFF7BAFE002008BD052008BD35
S11339303407FF1FF8B50746069E079C104850F849
S11339402750D6B1012085F824006A61AB61EE618D
S11339502E623846FFF782FF04280FD02835284608
S11339602146FDF741F90328F9D020B13846FFF785
S1133970D1FF0320F8BD0020F8BD0020F8BD00BF32
S11339803407FF1FF8B50546284B53F82040284B51
S113399053F82030226A002A3AD06268082A1CD8D8
S11339A030E0996B88B2DF62A26982B1266A022E86
S11339B004D194F840600EB1117008E01170A2694E
S11339C0511CA161000A5070A2690132A261226AED
S11339D0023A2262226A12B91AE04FF40037DA6A14
S11339E012F4003FDDD113E0996BD862A2691AB1D9
S11339F01170A2690132A261226A013A2262226A2A
S1133A0012B905E04FF40030DA6A12F4003FEBD14A
S1133A10E36913B12846FFF787FDE36923B9236AF5
S1133A2013B92846FFF73AFEF8BD00BF3407FF1F5D
S1133A30045F000008B5064B53F820301B68002BC8
S1133A4002DAFFF79FFF08BD00F0F0F808BD00BFE1
S1133A50045F0000F0B45F4B53F820305E4A52F824
S1133A6020201968C1F3C70011F0070F00F0A880E7
S1133A700130C0B2A4E09969002940F39D80012877
S1133A800AD11D691DB115F8011B1D6100E099687B
S1133A909D69013D9D6190E002281ED11E69BEB161
S1133AA0354615F801CB1D619F69013F9F61002FC9
S1133AB005DD71784CEA012101351D6104E0996846
S1133AC001F47F4141EA0C019D69013D9D6174E06F
S1133AD099690239996199686FE003282DD11E69AB
S1133AE036B3354615F8011B1D619F69013F9F617F
S1133AF0002F05DD767841EA062101351D6103E0DA
S1133B009D6805F47F4529439D69013D9D61002D14
S1133B1006DD1D6915F8016B41EA06411D6103E0EC
S1133B209D6805F47F0529439D69013D9D6144E03D
S1133B3099689D69033D9D613FE01E69002E36D062
S1133B40354615F8011B1D619F69013F9F61002FD8
S1133B5005DD767841EA062101351D6103E09D68A3
S1133B6005F47F4529439D69013D9D61002D06DDD6
S1133B701D6915F8016B41EA06411D6103E09D686A
S1133B8005F47F0529439D69013D9D61002D06DDF6
S1133B901D6915F8016B41EA06611D6103E09D682A
S1133BA005F07F4529439D69013D9D6105E09968C4
S1133BB09D69043D9D6100E099685163D46201E010
S1133BC04FF00074D16A11F0007F7FF454AFF0BC61
S1133BD0704700BF3407FF1F045F000070B5114B2E
S1133BE053F82050104B53F8206000242C732C61A0
S1133BF06C61EC61AC6130462146224600F0C6FAA5
S1133C0030462146224600F0AFFA30461B212246B8
S1133C1000F0CEFA30461321224600F0C9FA2C7186
S1133C2070BD00BF3407FF1F045F0000F8B50746EE
S1133C30604B53F82050604B53F820402368C3F383
S1133C40C70613F0070F01D00136F6B23846FFF766
S1133C5001FFE369002B7EDC84E0AB6BEA62012E9A
S1133C6009D1616919B10B70636901336361E36957
S1133C70013BE3616BE0022E17D1616989B10B70DE
S1133C806069411C6161E1690139E161002904DD78
S1133C901B0A4370636901336361E369013BE361B8
S1133CA055E0E369023BE36151E0032E22D16169EF
S1133CB0E1B10B706069411C6161E1690139E16145
S1133CC0002904DD190A4170616901316161E1690A
S1133CD00139E161002905DD61691B0C0B70636921
S1133CE001336361E369013BE36130E0E369033B72
S1133CF0E3612CE0616939B30B706069411C616157
S1133D00E1690139E161002904DD190A4170616941
S1133D1001316161E1690139E161002905DD616910
S1133D20180C0870616901316161E1690139E1616F
S1133D30002905DD61691B0E0B7063690133636142
S1133D40E369013BE36102E0E369043BE361E369A6
S1133D50002B02DC06E04FF40032EB6A13F4003F60
S1133D607FF47BAFE369002B03DC3846FFF736FFB3
S1133D70F8BDEB6A13F0006F0BD02B6B13F0006FE0
S1133D8007D04FF00063EB620D232371E388013306
S1133D90E380EB6A13F4002F0BD02B6B13F4002F8A
S1133DA007D04FF40023EB620D232371E388013322
S1133DB0E380F8BD045F00003407FF1F2DE9F00F16
S1133DC088B0069007910168002960DA4FF0FF344B
S1133DD000260120049003960296B446DFF8B890BA
S1133DE0DFF8B880834605962BE001FB03FA58F808
S1133DF0206059F82C7006FB07F5BAFBF5FA52451A
S1133E000BD3CAEB0205AC4207D92C46CDF814A05B
S1133E100491019D0395009E0296013102E05946EA
S1133E2001900096022901D8002CDED1009E0130B9
S1133E3001E0002066460F2801D8002CEFD10CF1D8
S1133E40010CBCF1030F01D8002CF2D1059E079F91
S1133E50BB1C069800EB83035A6822F00042049DC1
S1133E60691E42EAC1725A60596821F44031029FC6
S1133E703A0402F440320A435A60596821F00F01AF
S1133E80039800F00F020A435A60304600E0002015
S1133E9008B0BDE8F00F7047545F0000145F0000E5
S1133EA00368C3F30543012A01D10B4301E023EA6C
S1133EB00103026822F47C121B0403F47C131343F1
S1133EC00360704710B40368C3F380331BB1046804
S1133ED024F480440460046824F40054C94349036E
S1133EE001F4005121430160016821F48051D2435F
S1133EF0120302F480520A4302601BB1036843F4C4
S1133F00804303605DF8044B704700BF036823F4EB
S1133F100063C90201F400610B430360036823F4E6
S1133F208063920202F4806213430360704700BF0F
S1133F3010B50446036823F480430360036843F028
S1133F4001030360084BC362002383604FF0F04217
S1133F50C26002610363436301210A46FFF7D6FF8F
S1133F6044F20103236010BD00000A9A10B41368E0
S1133F70032B53D9102B02D90468012C50D0202BC9
S1133F8002D90468002C4DD00468002C28DA0231D0
S1133F9000EB8100416821F0F041013BDB0603F0B6
S1133FA0F0430B434360416821F0806113799B0621
S1133FB003F080630B434360416821F0007153793F
S1133FC05B0603F000730B434360416821F080718A
S1133FD093791B0603F080730B434360002022E0B7
S1133FE0023100EB8100416821F07841013B41EA54
S1133FF0C3634360416821F0806113799B0603F039
S113400080630B434360416821F0007153795B0680
S113401003F000730B434360002004E0062002E039
S1134020062000E006205DF8044B7047F0B49DF8CC
S113403010400568002D3CDA012C11D18D1C00EBD9
S113404085056F6827F44007960506F440063E434D
S11340506E606F6827F470471E03B6B23E436E600D
S1134060022C12D18D1C00EB85056F6827F44017D4
S1134070160506F440163E436E606F6827F47067B9
S11340801E0206F470663E436E60032C11D10231A9
S113409000EB8100416821F44021920402F44022A3
S11340A00A434260426822F0F0021B01DBB2134370
S11340B04360F0BC704700BF2DE9F04F85B002911A
S11340C003920E9E0268002A43DA244AB2FBF3FEEE
S11340D0CEEBCE084FEA08484FEA4E04B44224D34C
S11340E003990091029900221346FFF79FFF20468F
S11340F030E059F8274004FB0EFB5CF8214004FB38
S11341000BF4B44207D3C6EB040B5D4503D95D46FB
S1134110A0460B465246013101E00021BA460F2960
S113412001D8002DE5D1013708E04FF0FF350F230A
S113413003220027DFF82890DFF828C0032F01D8D6
S1134140002DEAD1039900910299FFF76FFF4046D1
S113415000E0002005B0BDE8F08F00BF00CA9A3B24
S1134160A45F0000645F0000036B23F08073090602
S113417001F080710B430363036B23F00073520659
S113418002F0007213430363704700BF036B23F410
S11341908033090401F480310B430363036B23F47C
S11341A00033520402F4003213430363704700BF28
S11341B010B4046B01238B4024EA03038A401343A5
S11341C003635DF8044B70470B784878000700F0F0
S11341D0E04040EAC3708B781B0403F47C1318435B
S11341E0CB78DB0603F0006318430B799B0603F0DE
S11341F080631843704700BF084B53F8203041F2E6
S113420021025A6000229A6030B9054A41F23C0307
S1134210D15821F48021D150704700BFB45F000011
S11342200070044038B5274B53F82040A568AD0F03
S1134230032D1FD8DFE805F002070E15A36843F02D
S11342404043A36016E0A36823F0404343F00043D7
S1134250A3600FE0A36823F0404343F08043A360CE
S113426008E0A36823F04043A36003E00B782370C5
S1134270013A013111F0030F06D0002AF6D103E010
S11342800B682360043A0431032AF9D8022A09D0BE
S1134290032A02D0012A0AD107E00B8823808B78F5
S11342A0237004E00B88238001E00B782370204600
S11342B000F04EF8A36823F0404343EA8575A560F7
S11342C038BD00BFB45F000010B40A4631B3154BCB
S11342D053F820300C7803F1047101F10B0008311C
S11342E040010460147B986820F0404040EA8470E8
S11342F09860507B9C6824F04054000700F04050C4
S113430020439860907B490188669068586001203A
S1134310486652681A600020486600E001205DF893
S1134320044B7047B45F000010B50B4659B130B967
S1134330064941F23C028C5844F480248C501946BE
S1134340FFF7C2FF10BD012010BD00BF0070044084
S113435000F104730B335B011B6813F0FF0302D0FD
S1134360012B0DD00EE08368C3F30173023BDBB273
S1134370012B02D8408880B27047008880B2704711
S1134380006870470020704700230380704700BF17
S1134390F0B403880026B44641F221070EE08C5D98
S11343A083EA0423644606E05D0013F4004F00D062
S11343B07D4001342B46072CF6D901369642EED3C4
S11343C00380F0BC704700BF03880B80704700BFB8
S11343D04FF0FF33036000234360704770B584B02F
S11343E004460E4601238DF8003003680193104BF8
S11343F0029300238DF80C308DF80D308DF80E30BB
S113440015466AB1FCF742FC00206946FFF78CFFB1
S1134410002031462A46FFF705FF0190FCF73EFCD9
S1134420019B236063681D44656004B070BD00BFD8
S1134430B71DC10430B583B004460D46426812F07E
S113444003020BD000238DF804308DF805308DF86D
S1134450063001A9C2F10402FFF7C0FF23682B60F4
S11344600020FFF7C9FE03B030BD00BF10B40346FF
S1134470816829B142684842824203D9002202E09D
S1134480002200E001220A48446810466AB15B68D1
S11344902268934206D30B44013B6268934203D9DA
S11344A0002002E0002000E001205DF8044B70478A
S11344B01004FF1F10B584B0044601A8FFF788FF5D
S11344C0626848F2CF339A4205D8A368134448F28D
S11344D0CC318B4205D801A81146A268FFF77EFFB4
S11344E011E001A81146C2F50342CC32FFF776FF72
S11344F06268A3681A4401A848F2D031A2F50342C5
S1134500D03AFFF76BFF01A803A9FFF793FF0398C5
S113451004B010BD436FB3F1FF3F07D1836FB3F114
S1134520FF3F03D1C36FB3F1FF3F03D042F6A203B1
S1134530C362704742F6A303C362704738B5124B97
S11345409B681C69E36A42F6A30293421AD004F101
S113455070052846FFF78AFF78B12846FFF7AAFFBF
S1134560E36F834204D042F6A103E362002038BD26
S113457042F6A003E362012038BD42F6A403E362DD
S1134580002038BD012038BD1004FF1F48F2040389
S11345901B6803604FF400431B680B60704700BF47
S11345A0054B9B681B6993F88E3013F0010F14BF01
S11345B000200120704700BF1004FF1F38B5064BD0
S11345C0DC691D46EB685B689847E368DB68002B91
S11345D0F8D020469847F5E71004FF1F38B5054684
S11345E00C46002001F090F8084B1C60084A156046
S11345F04FF40041074A916084F3088884F30988E2
S1134600A847002001F080F838BD00BF4809FF1F0B
S11346104C09FF1F00ED00E00F4B9B681B69421E15
S113462012F1030F09D80D4A904206D01A6982424A
S113463003D859690A44824208D85A6A824207D880
S11346409B6A1A44824205D80020704701207047B3
S113465000207047012070471004FF1FD904000098
S113466008B5FFF7D9FF034610B1FFF767FF03460C
S1134670184608BD2DE9F04F83B03C4B9B681D697B
S11346803B4C0AE095F88020134205D0E3685A6851
S1134690636920469969904718342368002BF1D147
S11346A04FF47A70FDF7DAFE044601A86946FFF775
S11346B06DFF01F0E1F9002839D10198FFF7D0FF2F
S11346C0002837D0FFF76CFF18B101980099FFF765
S11346D085FFB5F882904FF6FF73994501D14FF0ED
S11346E0FA0904FB09F9FDF79FFE06460F4623E08D
S11346F0B9F1000F0CD0FDF797FE801B61EB0701A9
S1134700A94208BFA04203D301980099FFF766FFAE
S1134710D34607E0DBF80C301B685846984788B945
S11347200BF1180BDBF80030002BF3D10BE04FF04A
S1134730000901E04FF000094FF0000B4C46002542
S1134740DFF82CA0D846B8F1000FD1D0084C06E011
S1134750A04503D0E3689B68204698471834236833
S1134760002BF5D1404603B0BDE8F08F1004FF1FC5
S11347708C6000005B4B1A6822F480621A605A69EC
S113478042F480625A61584A916A21F0807121F49E
S1134790014141F480719162196821F4006119604A
S11347A0596941F400615961D16A21F0807121F4A1
S11347B0014141F48071D162196821F400511960FA
S11347C0596941F400515961516B21F0807121F410
S11347D0014141F480715163196821F40041196069
S11347E0596941F400415961D16B21F0807121F480
S11347F0014141F48071D163196821F400311960D9
S1134800596941F400315961536C23F0807323F4E6
S1134810014343F480735364344B1A6842F0010239
S11348201A605A6942F001025A61314A116821F052
S1134830807121F4014141F480711160196821F003
S113484004011960596941F004015961916821F02A
S1134850807121F4014141F480719160196821F45F
S113486080711960596941F480715961116A21F0AC
S1134870807121F4014141F480711162196821F0C1
S113488080011960596941F080015961D36923F0AD
S1134890807323F4014343F48073D361154B1A6886
S11348A042F480421A605A6942F480425A61124AC0
S11348B0916B21F0807121F4014141F48071916385
S11348C0196841F480611960596941F48061596142
S11348D0936A23F0807323F4014343F48073936257
S11348E0704700BF00F00F400090044040F00F40BC
S11348F000A00440C0F00F4000C004402DE9F04384
S1134900BBB0FCF7BBF901F05FF86E4FBB681B68E6
S11349109847002000F0F0FFFDF75CFD07F1200050
S1134920FEF7BCFB3B681B689847FFF723FF00209A
S1134930022101F04FF901268DF89A6000248DF8C8
S113494099408DF89C608DF898408DF89B602046C6
S113495028A926AAFEF7C4FE4FF00809CDF88C90CA
S11349608DF891408DF890408DF892404CF250357E
S11349703AA941F8605D204625AAFEF74DFF20467E
S113498031462A4621ABFEF729FF204602212A465A
S113499021ABFEF723FF204603212A4621ABFEF775
S11349A01DFF494A1FAB1068516803C305230093D8
S11349B04FF0FF38CDF80480204621461FAA1DABD6
S11349C0FEF7B8FFBB681B699DF8772002F01F0251
S11349D0A3F89E208DF822608DF821408DF8246084
S11349E08DF820408DF8236002200AA908AAFEF75A
S11349F077FECDF814908DF819408DF818408DF895
S1134A001A403AA941F8D85D022007AAFEF704FF2C
S1134A10022031462A4603ABFEF7E0FE022001469F
S1134A202A4603ABFEF7DAFE022003212A4603AB33
S1134A30FEF7D4FE9E238DF87C3018238DF87D304C
S1134A4002250095CDF80480284621461FAA1DABF7
S1134A50FEF770FF89238DF87C3012238DF87D30AA
S1134A600095CDF80480284621461FAA1DABFEF709
S1134A7061FF8E238DF87C3020238DF87D300095E6
S1134A80CDF80480284621461FAA1DABFEF752FF2D
S1134A90BB685B689847FFF7EDFDF861036913B1E4
S1134AA01B6803B19847074BD869436913B11B6866
S1134AB003B19847034BDB681B6898473BB0BDE8DC
S1134AC0F08300BF1004FF1F205E000008B5FFF74D
S1134AD015FFFFF773FD00BF704700BFBFF34F8F93
S1134AE0044AD16801F4E061034B0B43D360BFF384
S1134AF04F8FFEE700ED00E00400FA0508B5FFF76C
S1134B00EDFF00BF08B5FFF7E9FF00BF08B5FFF7E9
S1134B10E5FF00BF08B5FFF7E1FF00BF024BDB680C
S1134B20DB680020186070471004FF1F431EDBB2CF
S1134B30102B08D8054BDB689B6800F10050013846
S1134B4003EBC00070470020704700BF1004FF1F34
S1134B5008B5094BDB68DB681B6A5BB10023037093
S1134B60054BDB68DB681B6A5B680BB1984708BDC3
S1134B70002008BD002008BD1004FF1F08B5044B29
S1134B80DB68D8680C300021142201F03EF908BD1E
S1134B901004FF1F10B584B0A0238DF80430002347
S1134BA08DF805308DF8063002228DF8072002902A
S1134BB00391044AD0694269946801A90C22A04770
S1134BC004B010BD1004FF1F2DE9F04182B0064669
S1134BD0884604781B4BDD68EF682046FFF7A6FF84
S1134BE03862EB681B6A03B31B680BB316480DF1FC
S1134BF00701FEF717FA0546E0B99DF807303BB107
S1134C00631E4FF4E75242FA03F313F0010F09D085
S1134C100C4BDB68DB681B6A1B68304641469847CF
S1134C2000200CE042F2117504E042F2107501E03C
S1134C3042F2107528462146FFF7ACFF284602B021
S1134C40BDE8F0811004FF1F3004FF1F10B582B0CF
S1134C5000238DF80730204BD8694369002B37D0E7
S1134C601D4AD268D268116801291ED05C68111DE2
S1134C7008320023A047034638B142F21272904230
S1134C8003D042F21372904223D1134AD268D268FD
S1134C909168F1B15068FFF797FF0346C8B90E4A0F
S1134CA0D268D2680121116013E00DF10700FFF70B
S1134CB04FFF034628B1084AD268D2680021116028
S1134CC007E0054AD268D2689DF80710116000E039
S1134CD00023184602B010BD1004FF1F08B5017868
S1134CE00020FFF757FF0A4BD86943691B699847AF
S1134CF0022000F009FDBFF34F8F064AD16801F48A
S1134D00E061054B0B43D360BFF34F8FFEE700BF59
S1134D101004FF1F00ED00E00400FA0510B504467E
S1134D20FCF766FF2178FFF735FF10BD10B5044688
S1134D30044B1B685B694068A16898472178FFF7BA
S1134D4029FF10BD1004FF1F10B50446FFF716FF1E
S1134D50074BDB68DA6861681161DB6808221A773F
S1134D6000202178FFF716FFFCF73CF910BD00BFC7
S1134D701004FF1F10B50446044B9B68DB680079E0
S1134D80A16898472178FFF705FF10BD1004FF1FA5
S1134D9010B50446FFF7F2FE074BDB68DA68A1683A
S1134DA01161DA6861685161DB6804221A770020B6
S1134DB02178FFF7EFFE10BD1004FF1F10B5044665
S1134DC0124BDB68D96800224A61D9680A61DB6842
S1134DD01B7F042B05D10D4B1B681B69984704B935
S1134DE004460A4BDB68DB682046197FFFF7D2FED6
S1134DF042F212739C4207D1044BDB68DB681B7FD1
S1134E00082B01D1FCF7A8F910BD00BF1004FF1F47
S1134E10F0B583B00446394BDB68DB681B6923B902
S1134E2000202070FFF7CAFF64E001230370334AB7
S1134E30D168C9680D694E6900210091D069426941
S1134E40576801A96A46B847074650B12B4BD86941
S1134E504369DB6898473846FFF7B0FF00232370A7
S1134E6048E0009931B942F21270FFF7A7FF00231E
S1134E7023703FE08D4238BF294600911F4BDB6809
S1134E80DB681A7F082A11D10198D8601B4BDB68B4
S1134E90DB689961FCF732F942F27D7398420ED0D7
S1134EA042F2747398420AD0074608E0134B1B6819
S1134EB09B683046019A98470746009B1E44009B16
S1134EC0ED1A05D13846FFF779FF0023237011E06E
S1134ED057B10A4BD8694369DB6898473846FFF7EE
S1134EE06DFF0023237005E0044BDA68D3681D616D
S1134EF0D3685E61002003B0F0BD00BF1004FF1F43
S1134F002DE9F0418AB00646334BDB68DB681B6948
S1134F1023B900203070FFF751FF58E001230370DC
S1134F202D4BDB68DC682769D4F81480E168237FA3
S1134F30202F34BF3D46202529B102A82A4600F07F
S1134F405BFF002418E0032B08D1234B1B685B682C
S1134F504046294602AA984704460CE0102B09D182
S1134F60637F00931D48414602AA2B46FEF7CEF903
S1134F70044600E00024A8446CB1174BD869436987
S1134F809D6802A900220123A8472046FFF716FFC7
S1134F90002333701BE07F1B0F4BD86943699C6867
S1134FA002A92A460123A04727B9FFF707FF0023D8
S1134FB033700CE020B1FFF701FF0023337006E0EB
S1134FC0054BDB68DA681761DB68C3F814800020DE
S1134FD00AB0BDE8F08100BF1004FF1F3004FF1FBA
S1134FE010B50446054B1B68DB684068A168E2689D
S1134FF098472178FFF7CEFD10BD00BF1004FF1FB6
S1135000F8B5044646688768C368194A1360194AA4
S1135010526843B1D1688B4207D31269013293427B
S113502005D8002504E0002502E0042500E004255D
S11350303046FFF7F1FA00B9042528462178FFF736
S1135040A9FDA5B90C4B1E60002000F05DFB0B4BC5
S11350501F60074B1B681BB183F3088883F309881F
S1135060054B1B6838469847002000F04DFBF8BDFF
S11350707C09FF1F1004FF1F7809FF1F7409FF1F1D
S113508038B504464068FFF7C7FA30B165680120B7
S113509000F03AFBA068A84700E004202178FFF75D
S11350A079FD38BD10B504460348211DFEF76CF99F
S11350B02178FFF76FFD10BD3004FF1F10B50446C3
S11350C00548616804F10C02A368FEF791F82178A1
S11350D0FFF760FD10BD00BF3004FF1F70B588B03E
S11350E0A7238DF8003000238DF801308DF80230AD
S11350F0551CEDB28DF80350019007E051F82300E0
S113510008AE06EB830444F8180C01339A42F5DC2C
S11351106A1C054BD86943699C6869469200002360
S1135120A04708B070BD00BF1004FF1F70B582B067
S11351300346002401940094084DAA6896680079F7
S1135140197A01AA6B46B047EB68DB681C610199C8
S1135150009A9208FFF7C2FF02B070BD1004FF1F4F
S113516010B584B0A3238DF8043001238DF80530E5
S113517000238DF8063002228DF807200290039157
S1135180044AD0694269946801A90C22A04704B07A
S113519010BD00BF1004FF1F10B50446FFF7EEFC5E
S11351A0074BDB68DA68A1681161DA6861685161EC
S11351B0DB6803221A770020A168FFF7D1FF10BD36
S11351C01004FF1F10B588B0AF238DF80030002302
S11351D08DF801308DF8023002238DF803300190F0
S11351E048B922FA03F302338DF80330029203A87C
S11351F000F002FE01E0002302939DF80320013237
S1135200044BD86943699C68694692000023A0470F
S113521008B010BD1004FF1F10B582B0044600236F
S113522000930193054861686A46A368FEF70AF88B
S11352306946A268FFF7C6FF02B010BD3004FF1F25
S113524010B584B0B0238DF8043001238DF80530F7
S113525000238DF8063002228DF807200290039176
S1135260044AD0694269946801A90C22A04704B099
S113527010BD00BF1004FF1F10B50446FFF77EFCED
S1135280094BDB68DA68A1681161DA686168516109
S1135290DA6810211177DB68227B5A770020A16835
S11352A0FFF7CEFF10BD00BF1004FF1F4368014A83
S11352B0D05C70478409FF1F08B5024B1B689847F0
S11352C008BD00BF8009FF1F10B504460079FDF733
S11352D069FAA36860680021984710BDF0B587B0EB
S11352E01023049300238DF814308DF81530594B96
S11352F09B681A69B2F89C204FF6FF718A4205D068
S1135300C2F30A025449A1F8542003E00021524A8E
S1135310A2F854101A69B2F89E204FF6FF718A421F
S113532005D0C2F30A024C49A1F8562003E07F21BC
S1135330494AA2F856101A6992F8992002F00F010E
S11353400F2920D00024444981F8524012F0080F5C
S113535019D0052481F850401B69B3F89A30190A12
S11353608DF80B10C3F342118DF80910C3F38201B9
S11353708DF80A1003F003038DF80C30C2F3021207
S11353808DF80820FFE7344C002384F852300423BE
S113539084F85030C5B2314B009301220192284663
S11353A004A92346FDF700F994F850305AB2052AAF
S11353B007D1042284F85020284602A9FDF7CAF830
S11353C007E05BB203EB8303284625491944FDF744
S11353D0C1F8214B93F8523033B101211E4B83F8AD
S11353E051102846FDF7A4FA284600214FF0FF3259
S11353F0FDF7BAF8002427464FF0FF3607E02846A9
S1135400394622463346FDF7BBF80134E4B2049A28
S11354109442F4D3104C002784F840700826666444
S11354202846314604F14002B4F85630FDF786F9B7
S113543028463146FDF772FA84F84870E664284637
S1135440092104F14802B4F85430FDF723F907B0F8
S1135450F0BD00BF1004FF1F8809FF1F6004FF1F79
S11354605060000010B50446164B1960836840680C
S113547002219847144B1A6822F004021A605A69F0
S113548042F004025A61114A916821F0807121F4BA
S1135490014141F480719160196821F08001196023
S11354A0596941F080015961D36923F0807323F471
S11354B0014343F48073D3616068FFF70FFF00205A
S11354C010BD00BF8009FF1F40F00F4000A0044042
S11354D02DE9F04782B081460E4617460024114D4F
S11354E04FF0080A05F1480816E03B1B082B02D8C8
S11354F0EB643C4602E0C5F84CA00834B5F85430DF
S113550099F8040000964FF47A72019209214246F8
S1135510FDF7DEF8EB6C1E44BC42E6D3002002B07B
S1135520BDE8F0878809FF1F10B504465A280AD140
S11355300122054B5A5408460449FDF70DFA044B61
S11355401B682046984710BD8409FF1FB95200000C
S11355508009FF1F08B5034B53F82000FDF7C4FB77
S113556008BD00BFD05E000038B50546214B53F896
S11355702040214B93F85230002B36D0236A1E4A28
S113558092F85120012A28D144F2080213420BD088
S113559013F40C4F08D120460121FDF70FFC002223
S11355A0154B83F8512020E0134A92F85030013B08
S11355B0DBB282F8503013F0800F03D004220E4B7C
S11355C083F850200C4B93F9501001EB81012846CD
S11355D00A4B1944FCF7BEFF07E013F44C4F04D008
S11355E0FDF7B0F92846FFF779FE2046FDF77CFB6E
S11355F038BD00BFD05E00008809FF1F5060000066
S11356000138042804D8DFE800F00D0507090B0071
S11356100548704705487047054870470548704776
S1135620054870470548704700A0064000C0064082
S113563000D0064000A00E4000B00E4000B006406E
S113564010B504464068FFF7DBFFFCF7EDFD60682A
S113565000F016F9A36860680021984710BD00BFE8
S113566010B50446054B19608368406801219847CA
S1135670606800F0D9F8002010BD00BFE009FF1FEA
S113568070B582B00446406801A900F0FDF808BB7B
S113569065682846FFF7B4FF0646284600F0DAF9A5
S11356A001463046019A0D4B1B68FCF77DFC60B93E
S11356B0A368606802219847084C23685A209847D9
S11356C02368A6209847012005E0606800F0ACF844
S11356D0002000E0002002B070BD00BFE009FF1F01
S11356E0F8B507460C4609E07868FFF789FF661CA1
S11356F094F90010FCF728FD2A463446551E002A6A
S1135700F2D10020F8BD00BF70B50646022802D0D1
S11357100020FDF7A9FB012E0ED115E004EB440394
S1135720DB002B44DB689A6822B104EB4400C00020
S113573028449047013401E000240E4D04EB440357
S1135740DB00EB58002BE9D176B9FBF79FFAFCF7A5
S113575063FEFBF7E1FA0022074B9A60012000F098
S1135760CBF800F043F962B6BFF36F8FBFF34F8FEE
S113577070BD00BF8C60000000ED00E02DE9F04139
S11357808046FCF751FE04460D46214B1A6801324F
S11357901A60204BD3E90023A21A65EB03031E49C8
S11357A00E6800279F4208BF964202D20122184B7E
S11357B01A60174B1B68013B062B24D8DFE803F063
S11357C00423230B14231800144BC3E90045144B82
S11357D0C3F8008017E01149D1E90023A21A65EB50
S11357E00303C1E900230EE00E4BC3E900450AE0C0
S11357F00C49D1E90023A21A65EB0303C1E9002394
S1135800404600F091F9034BC3E90045BDE8F0813F
S1135810EC09FF1F000AFF1FE409FF1FF809FF1F1F
S1135820E809FF1FF009FF1F10B5044600210C4BC7
S11358301960002200230B48C0E900230A48C0E98C
S113584000230A48C0E90023094B19600948FCF702
S113585005FE094B18602046084900F04BF910BDBD
S1135860EC09FF1FF809FF1FF009FF1F000AFF1FC3
S1135870E809FF1F80380100E409FF1F7D5700007D
S113588008B500F051F908BD10B50C46144B1B685F
S1135890072B21D1134B1B6898421FD1FCF7E6FD5F
S11358A0C0EB0010104B1A68104B1B681344B0FB7C
S11358B0F3F303EB83035B000D4AA2FB0313DB0941
S11358C005330C4AA2FB0313DB084FF4966202FB78
S11358D003F32360002010BD012010BD012010BD82
S11358E0EC09FF1FE809FF1FF809FF1FF009FF1F5C
S11358F0B5814E1BCDCCCCCC10B42E4B41F244021E
S11359002D49995041F238001C5844F4B0541C50AD
S1135910995041F24802995821F00F0141F00501D4
S1135920995041F204015A5842F440325A501A68CC
S113593022F440221A602148826C22F0807222F400
S1135940E06282641E4A2020507080241D48047046
S1135950585820F001005850AA231370D37803F04C
S11359601F03D3700B23137110235371937913F016
S1135970100FFBD1124A937903F00C03082BFAD1D0
S113598050220F4B5A711A46937903F00C03082BDB
S1135990FAD10B4A937913F0400FFBD02A22084B1B
S11359A01A701A46937903F00C030C2BFAD15DF8A4
S11359B0044B704700700440000033010090044021
S11359C0004006400050064008B5FCF7E5FC002204
S11359D0044B1A60044A41F23803D15841F4785117
S11359E0D15008BD00D0004000700440084B41F283
S11359F03802995821F4785199501A6822F00042DB
S1135A001A6041F20402995821F4E0219950704738
S1135A100070044041F24403044AD358C3F30363BF
S1135A200133034A1068B0FBF3F070470070044080
S1135A300004FF1F41F24403044AD358C3F3036331
S1135A400133034A1068B0FBF3F070470070044060
S1135A500004FF1F08B505280AD8DFE800F0030397
S1135A6006060606034B186808BDFFF7D3FF08BDFA
S1135A70002008BD0004FF1F114BDA6922F0807278
S1135A8022F4E06242F48072DA610E4A516921F034
S1135A9080015161DA6942F01302DA610023184689
S1135AA0084904E00A69C2F3C01210440133B3F593
S1135AB0FA7FF7D3F9288CBF00200120704700BF7C
S1135AC000B0044080F00F4008B5084B1B6C13F085
S1135AD0807F09D0064B1B6833B1002098474FF0F4
S1135AE0FF32024BC3F8A02008BD00BF00A0044051
S1135AF0080AFF1F88B9094B102283F83C234FF092
S1135B0080525A60064A136C23F0877323F480335F
S1135B1043F420231364034B1960704700E100E051
S1135B2000A00440080AFF1F70B94FF08052074BD1
S1135B30C3F88420064A136C23F0877323F480335C
S1135B4013640022034B1A60704700BF00E100E0B9
S1135B5000A00440080AFF1F704700BF032833D188
S1135B60012911D011B102291DD07047174B1A6CAD
S1135B7022F0807222F4E0621A645A6C22F080727D
S1135B8022F4E0625A647047104A136C23F0807365
S1135B9023F4E06343F4807313640D4B5A6922F4D5
S1135BA080325A617047094B1A6C22F0807222F4D9
S1135BB0E06242F440721A645A6C22F0807222F459
S1135BC0E06242F440725A64704700BF00B004407F
S1135BD080F00F4010B1022840D0704711B1022963
S1135BE01AD070473D4B1A6822F0807222F4E062AA
S1135BF01A605A6822F0807222F4E0625A609A684D
S1135C0022F0807222F4E0629A60DA6822F08072F4
S1135C1022F4E062DA607047304B1A6822F0807236
S1135C2022F4E06242F400721A605A6822F0807230
S1135C3022F4E06242F400725A609A6822F08072A0
S1135C4022F4E06242F400729A60DA6822F0807210
S1135C5022F4E06242F40072DA60704711B1022962
S1135C601AD070471E4B1A6D22F0807222F4E06243
S1135C701A655A6D22F0807222F4E0625A659A6DB8
S1135C8022F0807222F4E0629A65DA6D22F080726A
S1135C9022F4E062DA657047114B1A6D22F08072CB
S1135CA022F4E06242F400721A655A6D22F08072A6
S1135CB022F4E06242F400725A659A6D22F0807216
S1135CC022F4E06242F400729A65DA6D22F0807286
S1135CD022F4E06242F40072DA65704700C00440C6
S1135CE000A0044010B1012824D0704711B102294A
S1135CF00ED07047214BDA6C22F0807222F4E062FD
S1135D00DA649A6C22F0807222F4E0629A6470473A
S1135D101A4BDA6C22F0807222F4E06242F40072D0
S1135D20DA649A6C22F0807222F4E06242F4007227
S1135D309A64704711B102290ED070470F4BDA6C88
S1135D4022F0807222F4E062DA649A6C22F08072AB
S1135D5022F4E0629A647047084BDA6C22F0807295
S1135D6022F4E06242F40072DA649A6C22F08072E7
S1135D7022F4E06242F400729A64704700A0044086
S1135D8008B5084B1B6C13F0807F09D0064BDB6809
S1135D9033B1032098474FF0FF32024BC3F8A020E1
S1135DA008BD00BF00B00440200AFF1F70B50E4BB1
S1135DB00E4DED1AAD1000241E46AC4204D056F828
S1135DC0242090470134F8E700F084F9084D094B8A
S1135DD0ED1AAD1000241E46AC4204D056F824201F
S1135DE090470134F8E770BDF4600000F4600000EF
S1135DF0F8600000F460000010B50023934203D063
S1135E00CC5CC4540133F9E710BD02440346934209
S1135E1002D003F8011BFAE7704700005AA70000FC
S1135E200300060000000000F5110000311200001C
S1135E30791300008D1100006805FF1F0002015056
S1135E400000AAEAA11400001D180000C1160000F9
S1135E50A5140000B9160000B91400007D14000058
S1135E600000000015190000251900003119000078
S1135E700000000000000000411900007519000036
S1135E807D1900005D1A000000000000991B00004D
S1135E90511D0000211D0000B91D0000551E000009
S1135EA09D1C0000111E0000951E00009D1E000098
S1135EB0B11E0000F51E00000000000000000000FC
S1135EC0006006400070064000600E404C00000078
S1135ED0004002404D0000004B0000005000000054
S1135EE00000000000000800000010000000200076
S1135EF000004000000080000000000100000002DB
S1135F000400024000C0024000D0024000C00A4029
S1135F101A1B4100020000000400000006000000FB
S1135F2008000000100000002000000040000000F5
S1135F3080000000000100000002000000040000D6
S1135F4000080000001000000020000000400000D5
S1135F5000800000020000000300000005000000B3
S1135F600700000002000000040000000800000018
S1135F70100000002000000040000000800000002D
S1135F8000010000000200000004000000080000FE
S1135F90001000000020000000400000008000000D
S1135FA000000100010000000300000005000000E3
S1135FB007000000002003401D4D00000000000009
S1135FC02D4D00000000000099510000014F000019
S1135FD0914D0000114E0000E14F00000000000050
S1135FE0A5500000000000002D510000000000003A
S1135FF0494D0000114E0000015000000000000057
S11360008150000000000000DD4C00000000000092
S1136010754D0000000000000000000000000000BA
S1136020BD500000000000001952000000000000F4
S113603079520000014F0000000000000000000041
S1136040AD52000065540000C95200000000000079
S113605003070707030307070303030707010305F0
S11360600303010302030103010000000000000018
S1136070D1540000815600006156000041560000D2
S11360800000000000000000E156000001000000D4
S1136090000000005D5B000074600000846000008C
S11360A0445E00000800000000000000E55C000001
S11360B0406000006C600000445E000000000000CE
S11360C000000000000000000000000000000000CC
S11360D000000000F8B500BFF8BC08BC9E4670473D
S10F60E0F8B500BFF8BC08BC9E46704731
S10B60EC78A3FF7F010000000E
S10760F4350400006B
S10760F8110400008B
S11360FC00B4C404000000001407FF1FF406FF1FC3
S113610C905E00006C04FF1F285E00005004FF1F0B
S113611C000000008C600000000000000000000083
S113612C000000000000000000000000000000005F
S113613C000000000000000000000000000000004F
S113614C1D4B00004D4C0000B85F00005009FF1FB0
S113615C0000000029550000DD5200000000000082
S113616CFFFF0F00785E00000000FF1FFFFF0220FE
S113617CA85E000000000040FFFF0740605E0000C6
S113618C00F00F40FFFF0F40605E0000000000E0D5
S113619CFFFF0FE0605E0000000000000000000044
S10B61AC0000000000000000E7
S90304D91F
